:030000000219FDE5
:03000B000200AA46
:03002B0002015679
:03005B000202E5B9
:030073000202D2B4
:1000800002030406080C10182030406080040608A3
:100090000C10182030406080A0C00003070F1F0D17
:1000A0000D0403060D0502030202C2AFC0D0C0E07A
:1000B000206214E5256009E473E525F4F58AD2622F
:1000C000D0E0D0D0D2AF3285268AC262E526F46075
:1000D00029D0E0D0D0C293C295C297D2AF32C2939A
:1000E000C295C297206F0C206609740ED5E0FDE51D
:1000F0007B4290D0E0D0D0D2AF32758A00C28DD290
:100100006201F301B9306805206602D29301B9306B
:100110006805206602D29501B9306805206602D2D2
:100120009701B9C29230680A206607740CD5E0FDC9
:10013000D29301B9C29430680A206607740CD5E0E6
:10014000FDD29501B9C29630680A206607740CD5B5
:10015000E0FDD29701B9C2AFC2AD53E6EFC0D0C047
:10016000E0D2D3D2AFC2CEE52A6007207449152A67
:1001700021B77800790020742EE580307E01F430BC
:10018000E30278FF53DACF207E0343DA20307E0388
:1001900043DA10C2D8C271E580307E01F430E30248
:1001A00079FFC3E89970CB306103752A402074034E
:1001B000752A40885CD27020740DE52B6004152BE5
:1001C00021C743DA01C2D820700221DAA85C20617D
:1001D00002C27020740221D888227882B604038576
:1001E0002224C3E52594404002D26420CF0AD0E007
:1001F000D0D043E610D2AD32C2CF053A7802E52A1C
:100200006005307402152AC3E55C94014005755FF2
:10021000004124756000756900E55F2401F55F50B9
:1002200003755FFF7982B7020D306E1DC3E522941E
:10023000324016854C227982B7030E306E0BC3E52F
:100240002294324004798E8722C3E52395226008E8
:100250004004152341580523D8CA0569E569700291
:100260001569D56A63756A017805C3E569956B40C0
:1002700057C3E569956C50087801756A0302028CD2
:10028000C3E569956D50057801756A01C3E562950E
:1002900024401E7982B7040241BD206E1485246279
:1002A000E569046003856B69756A0175233C020288
:1002B000C8E5622850057562FF41BDF562E562043C
:1002C00070067560FF7569FFD0E0D0D043E610D2AC
:1002D000AD32C2AF53E67F7592FA7593FFC2607577
:1002E0009104D2AF32C2AF53E6EFC2ADC0D0C0E08E
:1002F000C0F0D2D3D2AFA8FBA9FCC2D83071026142
:100300004C53DACF207E0343DA10307E0343DA20E9
:10031000D271E580307E01F420E3026123882789D1
:1003200028A13153DACF207E0343DA20307E034305
:10033000DA10C2D8C271307402A11D7800E5803095
:100340007E01F430E302A11D885CA10553DACF20C1
:100350007E0343DA20307E0343DA10C2712061024B
:10036000812553DACF207E0343DA10307E0343DA4F
:1003700020C2D8D27188578958C3E89555F8E995B5
:1003800056F97B007E087A00C3E8948CE99400500B
:1003900005755B008117882178A2E6A8216055C306
:1003A000E894C8E994005008E4D2E4FB7A0A61F2C8
:1003B000C3E89468E994015008E4D2E3FB7A0F6142
:1003C000F2C3E894D0E994025008E4D2E2FB7A1E2A
:1003D00061F2C3E894A0E994055008E4D2E1FB7A05
:1003E0003C61F2C3E89498E994085008E4D2E0FB39
:1003F0007A787E00C3E89559FCE9955AFD30E70A02
:10040000ECF42401FCEDF43400FD755B00C3EC9AC0
:10041000ED9E5003755B018859895A85575585585B
:10042000567802A105C3E89527F8E99528F9307CAC
:100430000281E9307B0281E9307A0281E220750293
:100440008148E9FDE8FC8167E9C313F9E813F83056
:10045000790281E2E9C313F9E813F830780281E206
:10046000E9C313FDE813FC20612CC3EC941CED944C
:0E047000024002817EED701EC3EC94C850184D
:10047E000529E52970021529C3E529940A5002A120
:10048E001D755C00D270A11DE5296002152974004E
:10049E00207F037896E624FAFEE43400FFC3EC9E38
:1004AE00FCED9FFD50067800790081E9C3EC94FFC6
:1004BE00ED9400400678FF790081E9EC8572F0A496
:1004CE00C5F0A2F733F87900400302050578FF79ED
:1004DE0000020505E9C313F9E813F8307C0EE96054
:1004EE000278FFC3E81338F8E43400F9C3E894FF48
:1004FE00E99400400278FF885CD270206102A11D51
:10050E00741FF4552F4BF52FC274EB7002D2747515
:10051E002A40307403752A0A306102A13120740317
:10052E0053DAFE207403752B20D0F0D0E0D0D0D259
:10053E00AD43E61032790102056179030205617956
:10054E000A020561791E020561796402056179C8A6
:10055E000205617817E4D5E0FDD8FAD9F6227A14AF
:10056E007B780205887A107B8C0205887A0D7BB425
:10057E000205887A0B7BC80205887902E4C294D5FD
:10058E00E0FDD295D5E0FDC295D5E0FDD294D5E043
:10059E00FDE920E002D29330E002D297E573D5E078
:1005AE00FDE920E002C29330E002C2977496D5E0D6
:1005BE00FDD9C9EAF8D5E0FDD8FBDBBEC29422C353
:1005CE007C007D0075F00005F0EA33FAEB33FB504A
:1005DE00F6EB13FBEA13FAC3E9FFE8FEE89AF8E933
:1005EE009BF95004EFF9EEF8B3EC33FCED33FDD587
:1005FE00F0DFEDF9ECF822E889F08A20D2D4F8A9E0
:10060E00F07B0030F70B7BFFF42401F8E9F43400A3
:10061E00F9E88520F0A4ADF0F8E98520F0A4AFF05C
:10062E00FEED2EF974003FFA7C04C3EA13FAE913C7
:10063E00F9E813F8DCF48BF030F70AE8F42401F84B
:10064E00E9F43400F9E889F0C2D4F8A9F0227882EE
:10065E00B604030206FBC3E55C9419401EE52D5457
:10066E00067018206E3678057994E7146007780ABC
:10067E001460027812C3E54198401F306E098564FC
:10068E00627569FF756A01852224E4F544F545F526
:10069E0046F547F548C26E0206FBD26E7994E71412
:1006AE007013E523F43333F913F8E9540104F9E830
:1006BE0054FE0206EFE714147014E523F4333333BB
:1006CE00F913F8E9540304F9E854FC0206F7E5239C
:1006DE00F433333333F913F8E954070404F9E854C7
:1006EE00F8C39440F8E99400F98844894522C3E59B
:1006FE004113F9E54013F8C3E54498F8E54599F937
:10070E00500CC3E89480E994FF4016020733C3E807
:10071E00947FE994005003020733787F7900020733
:10072E0033788079FF8849894A22E5492546F8E5DC
:10073E004A3547F9854A20E4300701F43548FA3046
:10074E00E709C3EA94F04015020771C3EA940F500B
:10075E000302077178FF79FF7A0F0207717800792B
:10076E00007AF0C3E5249561500AC37401952450B4
:10077E000B02078FE54A20E70E02078FE54A30E7A6
:10078E0006884689478A482278A5E6FAC3E54933A2
:10079E00F8E54A33F9D105E930E70BC3E89480E96F
:1007AE0094FF4013E1C9C3E8947FE994005002E13D
:1007BE00C9787F7900E1C9788079FFE820E715C311
:1007CE00E52398F84009C3E8940140030207F07846
:1007DE00010207F0E8F424012523F840030207F094
:1007EE0078FF884B2278A6E6FAA847A948D105E9F2
:1007FE0030E70CC3E89401E994FF4016020824C3C5
:10080E00E894FFE99400500302082478FF7900026F
:10081E000824780179FFE920E715C3E54B98F840E5
:10082E0009C3E89401400302084B780102084BE823
:10083E00F42401254BF8400302084B78FF8824224C
:10084E0078FFC26420693D206A12D264C3E54194E8
:10085E000A4009C3E52594405002C26479A1E760BD
:0E086E0023E541601F74FF8541F0848539F059
:10087C00306A0375F005A4F8C5F0600278FFC3E890
:10088C0095645002A864886322C3E5409440E54116
:10089C009401E56350031401A6046002F563227809
:1008AC0083E6F520120F3D75E89012054375E8902C
:1008BC00E5E820ECFBA8BDA9BE120FE3756E307500
:1008CC006F00C3740013FD7430606613FC74302C1D
:1008DC00FC74003DFDECFAEDFBC3E89AE99B401477
:1008EC00E56E2430F56EE56F3400F56FEA2CFAEB0B
:1008FC003DFB80E5AE6EAF6FC3E56F13F9E56E138C
:10090C00F8C3E913F9E813F87A03C3E913F9E81308
:10091C00F8DAF7AA201A7009756E00756F000209D3
:10092C003D1AEA6008EE28FEEF39FFDAF88E6E8F7A
:10093C006F2275E890227883E6FFE5E820ECF7A8B3
:10094C00BDA9BE0570C3E57094084052757000E9EE
:10095C00FA79A0E76044EA7007E571601B02097838
:10096C00C3E895716010E5715006600C140209849F
:10097C000460F9020984E571F571C394A8401B75F4
:10098C0061C0C394054013756180C39405400B7519
:10099C006140C39405400375610075BB0122EFC330
:1009AC009401601F7430601BC3E894FFE9940350FA
:1009BC0012C3E8956EE9956F5009E561600C1561FD
:1009CC000209D6E561F460020561A861C3E52498CB
:1009DC005002A824C3E89562400AA862E562F4605C
:1009EC000385626188258826E570B4070375BB1EF4
:1009FC0022743279A787F0A4C5F0A2F733F8C3E8C4
:100A0C0095614002A86188228824882588268864FC
:100A1C00227540007541F022C2AF75C820A8CCA940
:100A2C00CDAA3A30CF010A75C824D2AFAB3BAC3C4F
:100A3C00883B893CC3E89BF8E99C206908F930673E
:100A4C00026130418DAD3D8A3DF9EA9DFA60047832
:100A5C00FF79FFAE3EAF3F8B3E8C3FA83BA93CC31A
:100A6C00E89EF8E99FF9C3E54113FBE54013FAE86A
:100A7C002AF540E93BF54150067540FF7541FF41B1
:100A8C00D7AA40AB41AC40AD417E047F02C3EB948E
:100A9C000440021E1FC3EB940840021E1FC3ED133B
:100AAC00FDEC13FCDEF7C3EA9CFAEB9DFBEF60094F
:100ABC00C3E913F9E813F8DFF7EA28FAEB39FB8AF4
:100ACC00408B4150067BFF8B408B41C3EB94025013
:100ADC0002D2673069047F0361027892E6FFC3E5B6
:100AEC0037948240110FC3E53794A040010FC3EF38
:100AFC00940640027F057E02E541C4540FF9E5419E
:100B0C00C454F0F8E540C4540F28F8C3E89EFAE941
:100B1C009400FB4009C3EA9402EB940050047A025F
:100B2C00E4FB617CAA40AB41EBC4FEEAC4540F4E1B
:100B3C00FCC3EA9CFAEB9400FBC3E813C313F8EA7A
:100B4C0028FAEB3400FB8A408B41C3EB9402400241
:100B5C00C2677802EBC4FE7B00EAC4540F4EFAC3A2
:100B6C00EA98FA4005C3940250027A027892E6FFA2
:100B7C00306002617C855192855293D26043E6804D
:100B8C00C3E49AF8E49BF93067028108E8FAE9FBC0
:100B9C00D3E913FDE813FC88518952C3EF94036029
:100BAC0038EF20E00DE82CF8E93DF9ECFAEDFB020A
:100BBC000BD1E828F8E939F9C3E82402F8E9340044
:100BCC00F97AFE7BFFC3EF9403400E8A538B548853
:100BDC004D894E8C4F8D50813C885389548A4D8B56
:100BEC004E8C4F8D503069127553F07554FF754F04
:100BFC00F07550FF7551F07552FF813CE8FAD3E85F
:100C0C0013FC8851C3EF94036020EF20E007E82C1D
:100C1C00F8ECFA8128E8282402F87AFEC3EF940352
:100C2C0040088A53884D8C4F813C88538A4D8C4F99
:100C3C00E568C3335002646BF56830600281467519
:100C4C003402D26043E680E52D54066034A840A9F6
:100C5C0041C3E913F9E813F8C3E913F9E813F830C1
:0F0C6C006904E92440F9C2AF53E67F759100C3D4
:100C7B00E498F594E499F595759104D26043E68078
:100C8B00D2AF22D265754300752000306C037520FE
:100C9B0040020CADD265754300752040306C037576
:100CAB00200078017901206720E52D54066002C2EF
:100CBB00657914E541C313700104F8C39414400221
:100CCB007814306904781B791B206010E543600CA5
:100CDB00306903D53404D26DA158914E0543E59E7E
:100CEB007005E59B020CF4E59A5440B52002A14235
:100CFB0030690908C3E89940011881D420650A08B6
:100D0B00C3E899400281AD81D4C265C2AF53E67F7F
:100D1B007591003067127594007595FE759104D22C
:100D2B006043E680D2AF81ADAE40AF41C3E49EF5E8
:100D3B0094E49FF595A127C3E5339401500281AD4F
:100D4B0030650281ADD802A15681D4C26DC2AF53BA
:100D5B00E67F759100855394855495759104854D67
:100D6B0092854E93D26043E680D2AFE52D54066058
:100D7B0008206A020533020D94306D0D206C0A2099
:100D8B0065071581158102162E2278003064053017
:100D9B0065027801E53775F007A4F9E5F028F5F061
:100DAB00E9A2F013A2F113A2F213F537C394785012
:100DBB0003753778C3E53795384008D266C293C2BE
:100DCB0095C297306002A1CE854F92855093D26029
:100DDB0043E68022207D19C2AF754202C294D292A3
:100DEB00306202D297D2AF759F33759E00020FE02F
:100DFB00C2AF754202C294D296306202D293D2AF86
:100E0B00759F33759E00020FE0307243207D20C228
:100E1B00AF754203900134757B10C297C296306256
:100E2B0004D295C132D294D2AF759E23020FE0C289
:100E3B00AF754203900134757B10C293C29230623E
:100E4B0004D295C152D294D2AF759E22020FE020EC
:100E5B007D17C2AF75420390010FC297306202D269
:100E6B0095D2AF759E23020FE0C2AF75420390017E
:100E7B000FC293306202D295D2AF759E22020FE061
:100E8B00207D16C2AF754204C292D296306202D256
:100E9B0095D2AF759E22020FE0C2AF754204C29687
:100EAB00D292306202D295D2AF759E23020FE03000
:100EBB007249207D23C2AF754205900123757B04D7
:100ECB00C295C294306204D293C1D8D292D2AF757C
:100EDB009F33759E00020FE0C2AF7542059001452E
:100EEB00757B40C295C294306204D297C1FBD296F7
:100EFB00D2AF759F33759E00020FE0207D1AC2AFF3
:100F0B00754205900105C295306202D293D2AF753E
:100F1B009F33759E00020FE0C2AF75420590011919
:100F2B00C2953062E8D297D2AF759F33759E00029F
:100F3B000FE0207D16C2AF754206C296D294306286
:100F4B0002D293D2AF759E23020FE0C2AF75420659
:100F5B00C292D294306202D297D2AF759E22020F08
:100F6B00E0307243207D20C2AF7542019001457580
:100F7B007B40C293C292306204D297E18AD296D25E
:100F8B00AF759E22020FE0C2AF754201900123752F
:100F9B007B04C297C296306204D293E1AAD292D25A
:100FAB00AF759E23020FE0207D17C2AF75420190F3
:100FBB000119C293306202D297D2AF759E22020FF3
:100FCB00E0C2AF754201900105C297306202D29325
:100FDB00D2AF759E23C26622900103757B00C2932C
:100FEB00C295C297C292C294C296C2622278807690
:100FFB00070876070876010876040876FF0876FF5F
:10100B00087607087602087601087601788C760157
:10101B000876000876B40876FF0876FF0876FF0896
:10102B0076030876FF0876010876FF0876250876A2
:10103B00D00876780876C80876040876FF0876011B
:10104B0008760008767A087610087601087601088B
:10105B0076000876FF087600227887E6FFC2727862
:0E106B0088C27DE630E102D27DC27E7889E641
:1010790030E102D27EC3EF94026008758E01D2730B
:10108900021091758E00C273227880E61490008058
:101099009378A5F67881E6149000809378A6F6787F
:1010A90086E61490008D9378A7F6789FE6F870018C
:1010B90008C3E8941140027811E82828F56B256BDC
:1010C900256B28F56C256B2828F56D7886E6F539AA
:1010D900C394025003753902789CE67538FFB4024F
:1010E900037538A0B4030375388278A3E614900019
:1010F9009A93F566120FE322227896E6FA7897E634
:10110900FB7888E6B40305C3EB940EFB307F047AC1
:10111900007BFFC3EB9AFCC3948250027C827572F8
:10112900000572EC8572F0A4C3E5F0947D40F222CB
:10113900D27F31021205527A007B007C10120548D9
:10114900E55C2AFA74003BFBDCF37C04C3EB13FB7C
:10115900EA13FADCF7FEC27F310222E5EF20E6034B
:101169007520000520903DFFE520146006901FFFC3
:101179001460009304600375EF1253D9BF7581C0E1
:1011890043FF8012054375EF0243B203E5B324021E
:1011990020E70DF521E5B120E0068521B343B10132
:1011A900120FE37580FF75A40075F1FE75D4F7750C
:1011B900900275A5FC75F2FC75D50075A0FD75A6A4
:1011C9000275F30275D60075B0FF75A70175F4FFB6
:1011D90075E241120FE3E4F8F6D8FD756801120FC4
:1011E900F812168578988673753001C2AF12055CBE
:1011F90012056C12055212057312055212057A1264
:1012090005521217A812055C12055C120557C2AFE8
:1012190078FA79FA308307D9FBD8F7021C001164F0
:1012290011923101310278988673120FE375881093
:1012390075890275C82475910475D84075A82275F9
:10124900B80275E690759B80759D00759A80759CAE
:101259000075D10E75BC5875BB0175BA1F75E8804C
:10126900120543D2AF1208AB75360053DACF207E90
:101279000343DA20307E0343DA1043DA01C2D8C2CD
:101289007112055CD2617B037A0CE55B70077A0CFD
:10129900DB03021217120552207003021217C270E3
:1012A900E55CC3940240E1E52F541F855E5DF55E60
:1012B900B55DD5DAD5C26153DACF207E0343DA2092
:1012C900307E0343DA10C2D8C27178A2E67008D220
:1012D90074E52F54E0F52FC27575290012055730B2
:1012E9007409C3E529940A4002D2751205487802A7
:1012F9003074027800C3E55C9840F0C2AF12056C07
:1013090012056C12056CD2AF12055C754C00120502
:1013190048788CE6C3940150030213EDE530C39479
:101329000150030213ED207435C3E55C94FF5003AB
:101339000213EDC2AF120581D2AF120557C3E55CA6
:10134900940150EFC2AF12056C12054D12056CD213
:10135900AF120557C3E55C94FF40E902182D7F05DC
:10136900D27F3102120557C2AFC27F3102AE5CC3D0
:10137900E55C947FD2AF4076120543C2AF12058176
:10138900D2AFDFDC3139C3EE94057897F612055CEC
:101399001216C71217B07F0AD27F3102120557C23F
:1013A900AFC27F3102AE5CC3E55C947FD2AF50E639
:1013B900120543C2AF12056C12054D12056CD2AF6E
:1013C900DFD63139EE24037896F612055C1216C77A
:1013D9001217DF1205573102C3E55C94FF50026111
:1013E9002F02182DC3E55C954C4003855C4C120512
:1013F9005778017988E7B403027805C3E55C98401A
:10140900026117C2AF120581120581120581D2AF9F
:1014190012055C753000E4F531F5320531E531F43A
:10142900703F0532789AE6781914601278321460A0
:101439000D787D14600878FA146003753200C3E5ED
:101449003298401D120FE3120543153275310078A9
:10145900998673C2AF120581D2AF78988673120547
:0F1469005712054DE52A700530740241177801BE
:101478002074027806C3E55C9840A1120557E52A56
:101488007003021217C2AF120FE3E4F522F523F539
:1014980024F525F526F567D2AF7885E6C333F565DB
:1014A800E4F544F545F546F547F548F570F52CF5AE
:1014B8002DF53775700875BB1E12054312093EE5F8
:1014C800E820ECFBA8BDA9BEE97001F888711209F3
:1014D8004275700875BB1E1164C2AF7561FF1209B1
:1014E800FD852261852262852263D2AF752201754E
:1014F8002401752501752601856069756A0178885A
:10150800E6B40307C27D307602D27DD268D269750F
:101518003300120F3D120F6C120A1D120A24120A10
:101528001D120A24120A1D120C9F12065C120D9538
:10153800120DDF120A24120C8E306E031206FC20E4
:10154800670312084E306703120895120D95120EA4
:1015580014120A24120C9F306E03120738120D95CC
:10156800120E8B120A24120C8E306E03120796127A
:101578000D95120EBA120A24120C9F306E03120730
:10158800F3120D95120F3D120A2412093E120C8E09
:10159800120D95120F6C120942120A2430692C851B
:1015A8006461856462856069756A0179187A0CC31B
:1015B800E533994009C269D26A8A350215D3C3E571
:1015C8005C9401400302152F021636306A1D206C08
:1015D8001AE535147006C26AD26BA12FF535C3E53A
:1015E8005C9401400302152F021636753600C3E5D8
:1015F8005F94014009856462856069756A0178FABB
:1016080079A4E760027803C3E55F98502130740439
:10161800E52A601A78F0306C058564617820C3E5A6
:1016280041985002A12F0536E55C6002C139753634
:1016380000C2AF120FE37887E6FE7602116478875E
:10164800EEF6E4F522F523F524F525F526F565757E
:101658002C00752D00D2AF120557120FE378A4E6BF
:101668006006D293D295D297307406E52A7002416B
:1016780017788DE6C39401400241F4811F901A0D3A
:101688007820121709E520B4A50CA3121709E52044
:10169800B45A030216A7120FF81216C70216C690FC
:1016A8001A0378807B0A121709A308DBF9901A0F2E
:1016B800788C7B19121709A308DBF9901A2822C223
:1016C800AF121748121722901A00740E12170EA3A1
:1016D800740612170EA3741512170E901A03788049
:1016E8007B0A12170DA308DBF9901A0F788C7B1967
:1016F80012170DA308DBF912175B121739901A2875
:1017080022E493F622E6438F01538FFD75EF0275AD
:10171800B7A575B7F1F0538FFE22438F02438F01AF
:1017280075EF0275B7A575B7F1901A0DF0538FFCD8
:1017380022901A0D74A5F10E901A0E745AF10E2209
:101748007A3079D07820901A40F109E520F709A37A
:10175800DAF7227A3079D0901A40E7F10E09A3DA45
:10176800F922AB74A875BB01027980BB02027981AA
:10177800BB03027982BB04027994BB05027983BB5F
:1017880006027986BB07027992BB08027987BB09F2
:1017980002799CBB0A027988BB0B027989E8F72297
:1017A8007C0512055CDCFB22C2AF12056C120573C6
:1017B80012057A12058112054D12056C1205731275
:1017C800057A12058112054D12056C120573120572
:1017D8007A120581D2AF22C2AF12058112057A12A0
:1017E800057312056C12054D12058112057A120552
:1017F8007312056C12054D12058112057A120573D4
:1018080012056CD2AF22AE74AF75C2AF12056C125E
:10181800056C12056C12054DDEF212058112054D9C
:10182800DFF8D2AF221217B01217A81217A87574D2
:1018380001757501757600110E7C05AD5C12055CAD
:10184800C3ED955C70F5C3E55C9401400AC3E55CA3
:1018580094FF403702187012176A1216C71217B091
:0F186800C2AF75EF121217A8DCD10576C3E57673
:101877009403500280C21217A80575E574149000EE
:101887009F93F808C3E57598500280A91217A8120C
:1018970017A80574C3E574940C50028095120FF8CD
:0B18A7001216C7C2AF75EF121217A88F
:0319FD0002116470
:101A00000E061507070104FFFF07020101A55A0191
:101A100000B4FFFFFF03FF01FF25D078C804FF01DA
:091A200000FF10010100FF00FFAE
:101A4000235467794B4631323041485623202020B9
:101A500023424C48454C4923463331302320202033
:101A60002020202020202020202020202020202076
:101C0000C2AFC2D353D9BF7581C043B20343FF8073
:101C1000752438752503B1C975EF0275E24043F1AB
:101C20000853A4F775D4FFD2837DFA780379E67C54
:101C300010752200752300901DD67B0675249875BB
:101C400025013083028142208308D8FBD9F9DCF7D3
:101C500081B4308308D8FBD9F9DCF781B4B189E4C9
:101C600093A3C39A6004DDC381B4DBDBB17B600264
:101C7000812B7B08E493FAA3B15CDBF87A30B15C8A
:101C8000752200752300B17BEAFCEBFDC3ED94FEE9
:101C9000400EB17B8A278B28ED30E0048A828B834B
:101CA000B17B7AC270D8C3ED94FE601350CEBD00F4
:101CB00025EC60097520007521FF0200008100A855
:101CC00027A9280809D804D90281D3B17FEA89AAB3
:101CD000F281C50D81A0C3ED94035049EDA2E092BD
:101CE000007AC5C3E5829400E583941C50902000DF
:101CF00010438F02438F0175B7A575B7F1F030001F
:101D00001FA827A9280809438F01538FFDD804D99C
:101D100002A12089AAE275B7A575B7F1F0A3A10DBC
:101D2000538FFC817C7AC1BD030CE493A3FAB140CC
:101D3000DCF8B138817C817EAA22AB23B15CEBFA5E
:101D4000EA6222752608C3E52313F523E52213F57D
:101D50002250066323A0632201D526EAB1C9B1C986
:101D600075260AEAF4200102D283300102C283B14F
:101D7000C9C3134002C201D526EB22B17FEAFB2082
:101D80008302A17F308302A184752608AE24AF258B
:101D9000C3EF13FFEE13FEB1CDB1C9C3EA13308315
:101DA000024480FA30E703632201C3E52313F523DD
:101DB000E52213F52250066323A0632201D526D91C
:101DC000E52265236523F52222AE24AF250E0FDE22
:101DD000FEDFFCD20122424C48656C693437316326
:041DE000F3100601F5
:00000001FF
